:020000020000FC
:100000000C9456000C94DB0D0C94DB0D0C94DB0D62
:100010000C94DB0D0C94DB0D0C94DB0D0C94DB0DC0
:100020000C94DB0D0C94DB0D0C94F6340C943135F0
:100030000C94DB0D0C94DB0D0C94DB0D0C94DB0DA0
:100040000C94DB0D0C94DB0D0C94DB0D0C94DB0D90
:100050000C94DB0D0C94DB0D0C94DB0D0C94DB0D80
:100060000C94DB0D0C94DB0D0C94DB0D0C94DB0D70
:100070000C94DB0D0C94DB0D0C94DB0D0C94DB0D60
:100080000C94DB0D0C94DB0D0C94DB0D0C94DB0D50
:100090000C94DB0D0C94DB0D0C943D0C0C94DB0DDF
:1000A0000C94DB0D0C94DB0D0C94DB0DA8950FEF7D
:1000B0000DBF0AE00EBF0E94100D0E948A027894C4
:1000C0000E943C010FEFC02E0E94FF000E94A6017B
:1000D0000C945F000590002009F0089500E0009363
:1000E000BD050C94F807E8EBFBE10E946A000716D7
:1000F00071F40E946A00061659F40E946A000516FF
:1001000041F431960591F491E02F099508953196C7
:10011000319630960C94750070EF60EF41E01881D5
:100120000E94C300013021F40E94B7000C948C009F
:10013000512F0E94B7001D30A9F03D2C18811D30B1
:1001400089F00E94C3003D1441F4762F652F512F92
:100150000E94B7004395433089F718810E94C3007D
:100160003D1409F008950E94B7000C94AD00DB1512
:1001700041F4CA1531F404E00093BD050C94F8076E
:100180000895219708951F9300271D3011F40C94B2
:10019000E6001F75103011F40C94D0001C3019F4D7
:1001A00001E00C94E700103112F40C94E7001B35C9
:1001B00012F00C94E70010341AF003E00C94E700FE
:1001C0001A3112F422F402E00C94E70004E0D02E7D
:1001D0001F910895CF3329F447E00E9428010C9421
:1001E000040148E00E94430140E20E944301412F84
:1001F0000E944301C3951DE018830C9404014EE353
:100200000E942801D5E0CFE30E944A01183011F383
:100210001F3701F31A3011F40C94040118831D30B8
:1002200069F0C03029F447E00E9428010C940401D1
:10023000CA95412F0E9443010C94040108950E9425
:1002400052028F93492F0E9428014F9101D00895A7
:100250000E941806B6FF0C9434012F930E94533469
:100260002F918823D1F3BF7B842F1F920E9481346A
:100270008823D1F71F9008954DE00E9428014AE09D
:100280000E94280108954D3019F40E943C01089500
:100290000C942801889500002F933F930E942E34E0
:1002A0003F912F919923B1F7182F08950E945B0178
:1002B0000E943C0108950091880A0023E1F34591D2
:1002C000442321F1483F21F40E9487010C945F01EF
:1002D000493F31F4159045910E94A1010C945F01B2
:1002E0004A3F21F40E943C010C945F014B3F51F4C2
:1002F000EF93FF93E4E7F1E20E945B01FF91EF913E
:100300000C945F010E9428010C945F010895EF9303
:10031000FF93112445914A3049F04C3039F04A3F5F
:1003200029F0493F19F013940C948A011A944CE374
:10033000141A1194169440E20E94A101FF91EF91CA
:1003400008950E9428011A94E1F70895D5E0CFE3BB
:100350000FEFA02E05E0B02E18810E94C3000230DE
:1003600011F40C949C060E943C01A1600C94B9010C
:10037000AE7F8DB78F3C28F408E00093BD050C9448
:10038000F8070E948C005D30F9F05B33E9F0032D33
:10039000023049F47F706F705F700E946D020E949E
:1003A000FA010C94B9017F756F755F75413039F4AE
:1003B000032D033021F40E94E6010C94B9010E9440
:1003C00073005D3009F00895A160089551545A31C9
:1003D0002AF005E00093BD050C94F807505CA0FFDF
:1003E00019F40E94FA010895F5E0E52F50810E946A
:1003F000FA0108950F93F4E0EC2D5083CA940C2D6C
:10040000033F28F406E00093BD050C94F8070F9114
:1004100008950F93C3940C2D00302AF007E0009349
:10042000BD050C94F807F4E0EC2D50810F91089570
:100430000E94090207E005175AF001E0503021F050
:10044000000F5A950C941E02502F0E94FA01089535
:100450000AE00093BD050E94F807703049F0705D16
:10046000472F0E942801603019F440E30E942801C0
:10047000603021F0605D462F0E942801505D452FBD
:100480000E942801089577276627545618F073951F
:100490000C9445025C595A5018F063950C944B0229
:1004A000565F0895982F9695969596959695905D9A
:1004B0009A3308F0995F8F70805D8A3308F0895F06
:1004C000089596FD975F9F7086FD875F8F70990FE7
:1004D000990F990F990F892B08957330B2F47230E8
:1004E00032F0663092F4653012F0563072F46623C2
:1004F00021F00AE0500F6A9581F7772309F40895F7
:1005000004E68894500F7A95C0F701E00093BD058A
:100510000C94F807E2ECFEE10E94560108950E9457
:100520003C01F4E0E4EFC091B905D091BA05FD17A4
:1005300011F4EC1731F040810E94430131970C9483
:1005400097020E943C010E943C01E0E4F1E20E941B
:100550005B015091B9057091BA05505071400E94ED
:10056000FA01572F0E9443020E942D02EEE4F1E2AD
:100570000E945B010E9409020E9443020E942D0218
:100580000E943C010895AE7F0E94B9010E940902B9
:100590000E9443020E942D020E943C0108950E9485
:1005A000B80144E20E9428010E940902852F0E949E
:1005B0001F010E943C010895AE7F0E94B9010E9474
:1005C0000902052F0E940902F5E0E52F0083089536
:1005D000A2FF0C949A03AE7F0E94B9010E94090207
:1005E000452E0E940902652F0E940902552EF5E052
:1005F000E52F6083A062A860AA7F0895F5E0E52D4D
:100600000081041519F003950083A06108950E94EC
:10061000B8010E940902052F0E940902501721F01B
:1006200055270E94FA0108955FEF0E94FA0108958C
:100630000E94B80150E000B605FE51E00E94FA01A8
:1006400008950E94B8010EEF0C1949F00E940902AA
:100650005F930E940902F52FEF910C9433030E94DF
:100660000902E52FFF2750810E94FA0108950E9498
:10067000B8010DEF0C1961F00E9409025F930E940E
:1006800009025F930E940902FF91EF910C944F03BE
:100690000E940902052F0E940902E02FFF275083C4
:1006A00008950E94B8010E940902052F0E940902C4
:1006B000509F1120F09921F4502D0E94FA010895C5
:1006C0000FE00093BD050E94F8070E94B8010E9448
:1006D00009025523F099B9F0052F0E940902652FF0
:1006E000771B59E0661F5A9551F0771F701B20F455
:1006F000700F88940C94720308940C947203562F14
:100700000E94FA01089501E10093BD050E94F807D7
:100710000E94B8010E940902052F0E940902500F91
:10072000F09918F00E94FA0108950FE00093BD05BA
:100730000E94F8070E94B8010E940902052F0E943A
:100740000902501BF0991BF00E94FA01089500E184
:100750000093BD050E94F8070E94B8010E9409029B
:10076000052F0E94090250230E94FA0108950E9459
:10077000B8010E94090256950E94FA0108950E944C
:10078000B8010E940902550F0E94FA0108950E94C3
:10079000B8010E940902052F0E940902502B0E94F5
:1007A000FA0108950E94B8010E940902052F0E94D3
:1007B000090250270E94FA0108950E94B8010E9480
:1007C000090250950E94FA0108950E94B8010E9402
:1007D000090251950E94FA01089551E00E94FA0120
:1007E00008950E94B8010E940902052F0E94090283
:1007F00050170C9403040E94B8010E940902052FAF
:100800000E940902051750E042F739F30E94FA01ED
:1008100008950E94B8010E940902552309F0A260C0
:1008200008950DB70E5F0DBF0895A46008950E944E
:10083000B8010895B260089598810E94B700888138
:100840000E946102582F0E94FA010E94B7000E9484
:10085000B80108950E94B8010E940902CF93DF9366
:10086000D0EAC9EFCA950000E9F7DA950000C9F7A8
:100870005A95B1F7DF91CF91089555270E94FA015B
:100880000E94B8010E94090201E005172AF0F098C1
:1008900050FF0895F09A08950CE00093BD050E9462
:1008A000F8070E94B8010E940902452FF4E0E4EF26
:1008B0008091B9059091BA050C946904F91711F467
:1008C0008E1708F500810D3019F031970C945E04F5
:1008D0003197552766277727F91711F48E1798F463
:1008E00010810E94C300023031F4762F652F512F02
:1008F00031970C946C047F706F705F700E946D0272
:100900004517E1F6089509E00093BD050C94F8073A
:100910000E945104DF2FCE2F08950E945104A06C35
:100920000895B2FF0C949604B1600895B2600895E2
:100930000E94B8010E940902452F0E9428010895D3
:10094000889500002F930E9453342F918823C1F380
:100950002F930E942E342F91582F533009F4B260F8
:100960000E94FA0108950E94B8010E94090208E05D
:1009700040E3551F08F441E36BDC0A95C9F70E9478
:100980003C01089504EB5091BE05579508F450279B
:100990005093BE050E94FA010895D4E0C4EF0FEF12
:1009A000C02EA1600E941806A5FF0C94DA046C2EDC
:1009B0007D2EAF7DA4FF0C94E004D72DC62DAF7E15
:1009C000A6FF0C94E804D093BC05C093BB05AF7B95
:1009D000A7FF0C94EF04DF2FCE2FB460AF77B0FFEA
:1009E0000C94F704C091BB05D091BC05BA7FB1FF50
:1009F0000C9401050E941106C091B905D091BA0569
:100A0000BD7F0091BA05D01721F40091B9050C17EC
:100A1000A0F418810E94C300A1FF0C9414050430B7
:100A200019F021970C94CF04AD7F023019F421976F
:100A30000C94CF040E94B901B2CF0895F4E0E4EF22
:100A4000F093BA05E093B9050FEFC02EAA27BB2794
:100A5000F1E0E0E000E00193F430E8F3E43FD9F79F
:100A6000F5E0E0E400E00193F530E8F3EA35D9F78A
:100A70000E943C01EAE7FEE10E9456010895E0E889
:100A8000F0E20E945B01EAEAF0E20E945B0100E111
:100A9000202EF4E0E4EF8F2F0E941F018E2F0E9482
:100AA0001F014AE30E94280140E20E942801F13020
:100AB00011F4E030D9F080810E941F0140E20E94D1
:100AC000280131972A9481F40E943C018F2F0E94C3
:100AD0001F018E2F0E941F014AE30E94280140E25D
:100AE0000E94280100E1202E0C9457050E943C0131
:100AF0000E943C01E6ECF0E20E945B018091BA05A5
:100B00000E941F018091B9050E941F010E943C01B3
:100B1000E0E8F0E20E945B010E943C010895E0E8F9
:100B2000F0E20E945B01EAE9F0E20E945B0100E171
:100B3000202EF3E0EFEF8F2F0E941F018E2F0E94D7
:100B40001F014AE30E94280140E20E9428010F93FE
:100B5000E03000E0F0070F91F1F0F2BDE1BDF89A4E
:100B600080B50E941F0140E20E94280131972A941B
:100B700081F40E943C018F2F0E941F018E2F0E9442
:100B80001F014AE30E94280140E20E94280100E17F
:100B9000202E0C94A7050E943C01E0E8F0E20E94A0
:100BA0005B010E943C010895E0E8F0E20E945B01D5
:100BB000E6E8F0E20E945B0100E1202EE0E4F5E0CF
:100BC0008F2F0E941F018E2F0E941F014AE30E9457
:100BD000280140E20E942801EA35D1F081910E946B
:100BE0001F0140E20E9428012A9481F40E943C01E6
:100BF0008F2F0E941F018E2F0E941F014AE30E9427
:100C0000280140E20E94280100E1202E0C94EC050E
:100C10000E943C01E0E8F0E20E945B010E943C017E
:100C200008950E946E34E8E3F1E20E945B010895AA
:100C30002F930E9453342F91882389F02F930E9481
:100C40002E342F91082F033111F4B06408952F939F
:100C50000E942E342F91082F033009F4B2600895BA
:100C6000DF93D4E0DA950000E9F7DF910895DF9390
:100C7000D8E2DA950000E9F7DF910895CF93DF938A
:100C8000D0EAC3EFCA950000000000000000D1F7D1
:100C9000CFEFCA95000000000000D9F7CCEFCA954D
:100CA0000000000000000000D1F716F06894E9CFC2
:100CB000DA95E89431F7DF91CF910895D5E0CFE34D
:100CC000552788279927BF7D1881CA9583951D30A0
:100CD00051F00E94C300023041F0B0620130A1F334
:100CE00093950C946406092F0895B5FF53950C94C1
:100CF000640604E00093BD050C94F80702E000933D
:100D0000BD050C94F8070BE00093BD0571C17F7021
:100D10006F705F700E946D020895D5E0CFE3E03000
:100D200069F308810083319721970D30C1F7F09363
:100D3000BA05E093B90508950E945E06543018F78D
:100D40008091B9059091BA05943021F4843F11F453
:100D50000C940B07D5E0CFE3552766277727CA15F4
:100D600042F218810E94C300023031F4762F652FC1
:100D7000512F21970C94AF060E948706452EE091D3
:100D8000B905F091BA05B77FBF7E7727662755274B
:100D900055243196F43011F4E53F69F010810E943A
:100DA000C300043041F0023081F75394562F672F6F
:100DB000712F0C94C906052D033031F05394562F32
:100DC000672F70E00C94DB06B4FD0C94EA06B0616A
:100DD0000C94C5060E9487064516F1F118F4B86018
:100DE0007F2E6E2EF43029F4E53F19F4B3FF0C94F6
:100DF0000B07B3FF0C940007541538F40C945607F6
:100E0000F43019F6E53F09F60895F43021F4E53F92
:100E100011F40C9456070E945E06003009F4089500
:100E2000D5E0CFE3E091B905F091BA05F13021F4B6
:100E3000E03011F40C942707088100833197219743
:100E40000D30A1F7F093BA05E093B905089502E0DB
:100E50000093BD050C94F8073197EF01D13021F4D0
:100E6000C03011F40C947906088121970D30B1F748
:100E70000E2F0C1B8091B9059091BA05800F8093BD
:100E8000B90518F493959093B905D13011F4C03099
:100E900031F008810083219731970C9445070E9417
:100EA0005E06003011F00C949C0608950E945E06C8
:100EB000003071F10091BA05013029F40091B905B3
:100EC0000050081720F2E091B905F091BA05DF2F24
:100ED000CE2FC81BD040D093BA05C093B905F715E3
:100EE00021F4E61511F40C947B0700810883219608
:100EF00031960C946F07D5E0CFE3F72DE62D3197AF
:100F0000088100830D3021F0319721970C948007E0
:100F10000895D4E0CFEFE091B905F091BA05CE1B6A
:100F2000DF0BF3E0EFEFEC17FD072CF4E2EEF0E25D
:100F30000E9456010895E2E0F1E20E9456010FEF8F
:100F4000C02E5091B9050E94FA015091BA050E9435
:100F5000FA01D4E0CFEFF3E0EFEF0881F9990C94B8
:100F6000AE07F2BDE1BD00BDFA9AF99AD13011F495
:100F7000C03051F031970F93E03000E0F0070F914F
:100F800019F021970C94AD070895E4E2F1E20E9474
:100F900056010E941E05D4E0CFEFEFEFF3E0F99980
:100FA0000C94CF07F2BDE1BDF89A00B50883D130AB
:100FB00011F4C03021F0319721970C94CF070DEF39
:100FC000C02E0E9409025093BA05F52F0E94090213
:100FD0005093B905E52F0F93EF3F04E0F0070F9111
:100FE00031F4E4E1F1E20E9456010E941E050895E9
:100FF0000E943C010091BD05000FE4E2F0E1E00F2A
:101000000591F491E02FEE1FFF1F0E945B010FEF8F
:101010000DBF0AE00EBF0FEFC02EA0E0B0E00E94AF
:101020003C014DC8BE10CF10EB10FA1018112E1154
:10103000451164118E11B811D211EB1102121B125D
:1010400034124712541262126D127B128B129C12D0
:1010500055270E94FA010E94B8010E94090201E08E
:101060000517A2F00CE050FD08E40093B800409A88
:10107000419A00270093B90000950093BB0004E05B
:101080000093BC0004E90093BC0008950CE00093B9
:10109000BD050E94F8070091BC0002FF0C947A087D
:1010A0000E94B8010E9409025093BB0005E800931A
:1010B000BC000091BC0007FFFCCF0091B900087F85
:1010C000083111F0003441F45091B900569556950D
:1010D00056950E94FA010895003239F0083429F03B
:1010E00002E10093BD050E94F80704E10093BD05ED
:1010F0000E94F80703E10093BD050E94F8070091E4
:10110000BC0002FF0C94AA080E94B8010E940902C8
:101110005093BB0005E80093BC000091BC0007FFA2
:10112000FCCF0091B900087F083241F45091B9001A
:101130005695569556950E94FA010895003329F068
:1011400002E10093BD050E94F80704E10093BD058C
:101150000E94F80703E10093BD050E94F807009183
:10116000BC0002FF0C94DD0851E00E94FA010E94CD
:10117000B8010E94090201E0051722F104EC50FFBA
:1011800004E80093BC000091BC0007FFFCCF009175
:10119000B900087F003529F45091BB000E94FA0184
:1011A0000895003529F002E10093BD050E94F8077B
:1011B00004E10093BD050E94F80703E10093BD051B
:1011C0000E94F8070CE00093BD050E94F80700910B
:1011D000BC0002FF0C94FE0804EA0093BC000091DE
:1011E000BC0007FFFCCF0091B900087F083009F46C
:1011F000089502E10093BD050E94F80703E1009302
:10120000BD050E94F8070091BC0002FF0C94140970
:1012100004E90093BC000FEF0093BB00089502E1C6
:101220000093BD050E94F80703E10093BD050E94ED
:10123000F8070091BC0002FF0C9432090091BC0039
:1012400004FF0C94260950E80C942F090091BC006F
:1012500007FFFCCF5091B9005695569556950E94C0
:10126000FA01089503E10093BD050E94F80752E0DA
:101270000E94FA010E94B8010E94090203E00517CA
:101280004AF0550F550F0E94A8090CB5037F052B96
:101290000CBD08950DE00093BD050E94F8070E9463
:1012A000B8010E94090201E0051752F00CB5006276
:1012B0000CBD50FD0C945F090CB50F7D0CBD08955D
:1012C0000CE00093BD050E94F8070E94B8010E943F
:1012D000090207E0051782F0052E53700CB5087F50
:1012E000052B0CBD0DB501600DBD02FC0C947B09F6
:1012F0000DB50E7F0DBD08950AE00093BD050E9457
:10130000F8070E94B8010E94090228980000000016
:101310005EBD0DB407FE0C9489095EB5089528984A
:10132000000000005EBD0DB407FE0C9493095EB58D
:101330000E94FA01089551E00E94FA010E94B8014A
:101340000E940902289A50FD0C94A7092898089534
:1013500004B1076004B905B1016005B901E50CBD30
:101360000DB50E7F0DBD0895009164000E7F0093B2
:10137000640000E000937B0055270E94FA010E9460
:10138000B8010E94090200917C00007E60917B0000
:101390006F7D60937B0056FF0C94D10960917B00B8
:1013A000606260937B005F71052B00937C0007EC0B
:1013B00000937A0000917A0006FD0C94DA0907EC9C
:1013C00000937A0000917A0006FD0C94E209509196
:1013D00079000E94FA01089555270E94FA010E949F
:1013E000B8010E94090201E005175AF000917C0043
:1013F0000F73006250FD0C94FE09006C00937C009A
:1014000008950CE00093BD050E94F8070E948A0A27
:10141000EF5DFF4F50810E94FA0108950E948A0AF1
:10142000EF93FF930E94B8010E940902FF91EF9190
:10143000EF5DFF4F508308950E948A0AEF93FF9358
:101440000E94B8010E9418020E940902FF91EF91C8
:10145000EF5DFF4F0C948F0A0E948A0AEF93FF936F
:101460000E94B8010E9418020E940902FF91EF91A8
:10147000EF5DFF4F0C94930A0E948A0AEF93FF934B
:101480000E94B8010E940902FF91EF91EE5DFF4FAB
:10149000508308950E948A0AE05EFF4F50810E94A7
:1014A000FA0108950E948A0AEF93FF930E94B801FF
:1014B0000E9418020E940902FF91EF91EE5DFF4F1A
:1014C0000C948F0A0E948A0AEF93FF930E94B8013E
:1014D0000E9418020E940902FF91EF91EE5DFF4FFA
:1014E0000C94930A0E948A0AEF93FF930E94B8011A
:1014F0000E9418020E940902FF91EF91E05EFF4FE7
:101500000081052350E000230FB601FC51E00E944A
:10151000FA01089503E05154509FF00108950081AD
:10152000052B0083089550950081052300830895BD
:101530000E94B80101E80093800009E00093810057
:10154000002700938200259A0E9409020027009339
:1015500089005093880008950E94B80103E8009321
:10156000800009E000938100002700938200259A03
:101570000E940902052F0E940902509389000093DE
:1015800088000895002700938000089555270E9441
:10159000FA010E94B8010E94090207E005178AF0CB
:1015A0000091BF05087F502B5093BF050027009383
:1015B0006F0006BB009382000093800000938100BF
:1015C00008950AE00093BD0513DD51E00E94FA0181
:1015D0000E94B8010E94090201E005174AF000913B
:1015E000BF050F7750FF01C000680093BF05089545
:1015F0000CE00093BD05FCDCCF93DF9366275527F5
:1016000056BB6093850050938400B09A0091BF054B
:10161000702F7078C894771F771F76600770E3E1AA
:10162000FBE0E00F09947AC006C005C004C02AC0E0
:1016300029C028C04FC0033008F005E07093810036
:101640006093850050938400D0E1C3EFCA950000F9
:10165000000000000000D1F7CFEFCA9500000000A5
:101660000000D9F7CCEFCA95000000000000000090
:10167000D1F716F06894E9CFDA95E89431F70A9536
:1016800019F74CC00350033008F005E07093810057
:101690006093850050938400D0EAC3EFCA950000A0
:1016A000000000000000D1F7CFEFCA950000000055
:1016B0000000D9F7CCEFCA95000000000000000040
:1016C000D1F716F06894E9CFDA95E89431F70A95E6
:1016D00019F724C0709381006093850050938400B3
:1016E0000AE0D0EAC3EFCA95000000000000000045
:1016F000D1F7CFEFCA95000000000000D9F7CCEF7A
:10170000CA950000000000000000D1F716F06894B0
:10171000E9CFDA95E89431F70A9519F750918400EA
:1017200060918500002700938100B09908C0C9E549
:10173000D5E068830E94FA01DF91CF910895DF918F
:10174000CF910EE00093BD0553DC0E94B8010E94CA
:101750000902152F88940E94BD0B08950E94B801BC
:101760000E940902152F08940E94BD0B08950E9443
:10177000E70B512F0E94FA01089504B1077E04B9C6
:1017800005B1086105B979E01C9B0C94C40B2D9A36
:10179000259810F02D98259A2C98249A0E94080CD0
:1017A00024982C9A0E94080C1C990C94CC0B20F0C5
:1017B0002D9A25980C94DE0B2D98259A1C9B0C9441
:1017C000DE0B25982D9A111F7A95F1F6089504B134
:1017D000077E04B905B1086105B979E01C990C943C
:1017E000EE0B88941D9B0C94FD0B08942C98249A66
:1017F0001D990C94F80B0C94020C2C98249A1D9BA8
:101800000C94FF0B24982C9A111F7A9539F70895A0
:1018100080E590E59A95F1F78A95D9F70895CF93E9
:10182000DF9355270E94FA010E94B8010E94090225
:101830000517F2F050FD0C94290C0E94F20CC3EC39
:10184000D5E00993099308835D9A5598DF91CF916C
:101850000895C7E5D5E00E94690C00270093C605EE
:10186000559A5D980E94CC0CDF91CF9178940895A1
:101870000CE00093BD050E94F8077F937FB77F932C
:101880006F935F93EF93FF93F5E2E091C60550915C
:10189000C3056091C4057091C505E50EF61EE71FEE
:1018A0005491E093C60550FF0C94600C00005D9AC3
:1018B000FF91EF915F916F917F917FBF7F9118951D
:1018C0005D98FF91EF915F916F917F917FBF7F91C5
:1018D0001895C7E5D5E077276627552700EF102E26
:1018E000088001200294002049F080E0581F90E019
:1018F000691F00E0701F0A940C94730C09901294F5
:101900000120002049F089E9581F99E9691F09E180
:10191000701F0A940C94810C088012940120029488
:10192000002049F08CE5581F9FE8691F02E0701FF6
:101930000A940C94900C099012940120002049F014
:1019400089E8581F91E4691F00E0701F0A940C9405
:101950009E0C0880129401200294002049F08DE82A
:10196000581F96E0691F00E0701F0A940C94AD0C9C
:10197000088012940120002041F087EA581F90E06F
:10198000691F00E0701F0A94B1F75093C30560937C
:10199000C4057093C5050895009165000F7E0093FE
:1019A0006500002709BB0093BE000093C0000093B0
:1019B000C1000093CF000093D0000093C2000093B9
:1019C000C3000093C4000FE90093D10000E000932E
:1019D000C00001E00093C100009172000064009318
:1019E00072000895F894002709BB0093C00000938B
:1019F000C1000093BE000093D0000093CF0000937D
:101A0000C2000093C3000093C400009172000F7BDA
:101A100000937200009165000061009365000895D5
:101A2000A89504B7007004BF00916000086100939E
:101A300060000070009360000E941D3406E204B94B
:101A400000E005B900E007B900E008B908E00AB90C
:101A500000E00BB900E00DB900E00EB900E000BBFA
:101A600000E001BB00270093BF050EBBF09A54EBCA
:101A70000091000105270093BE050E9403340E94D7
:101A80006E340E94E5348AE00E943E068A95E1F7B2
:101A90000E942B348823E1F301E003BF5F9A0E9488
:101AA00037064F990EC05F980E94C5070E94CD046B
:101AB0000E943C010E943C01EAE7FEE10E945601BF
:101AC00008952F930E9453348823E1F32F910E94AD
:101AD0001E050895E3E0F0E009E007BF04910695D4
:101AE0000370003019F4E0E0F8E314C0013019F499
:101AF000E0E0FCE30FC0023019F4E0E0FEE30AC0CE
:101B0000033019F4E0E0FFE305C00BE00093BD05EE
:101B10000C94F807EF93FF9308E0102EEE1FFF1FC1
:101B200005910F3F19F0003009F007C01A94C1F772
:101B300005E10093BD050C94F807E8E5F1E20E9489
:101B40005B01FF91EF918F2F0E941F018E2F0E944A
:101B50001F010E943C010E943C0111240E94E534B7
:101B60000AE00E943E060A95E1F70091E80000FFB6
:101B7000FCCF0E941D34F8941DBA109268001CBC62
:101B800010BE1FBA10926E0010926F00109271007A
:101B9000109272001092C9001092BC0010927A004C
:101BA00014B817B81AB81DB810BA15B818B81BB8B9
:101BB0001EB811BA099418954C4953208F025255FA
:101BC0004E20CD045052494EC30250525820CF02ED
:101BD00050524220B304464F522015044E455854EB
:101BE000FE0253495A20A3024E4557201E0550506D
:101BF0000B20880350500D209A0350500A205103A7
:101C000050500F206503414F56203D04454D495427
:101C10009804501A1D20DC0250501D20E802501C70
:101C20001E20070350501E20FB0350501C20F103C0
:101C300050494620090450544F20170450500420A6
:101C40001C04454E44201A04414E4420AC034C531E
:101C50005220B7034C534C20BF03504F5220C703B0
:101C6000584F5220D203434F4D20DD034E454720AD
:101C7000E503524E4420C20444454C412A04474FD8
:101C8000544F8804474F53558D0452455455910481
:101C90005448454E11044B455920A00441434F2060
:101CA00018035341564589074C4F4144C5075045D9
:101CB000454B2103504F4B4537034F4442200E0AFA
:101CC00049444220060A534442201C0A434442200D
:101CD0002C0A4F5042203C0A53424220520A4342AF
:101CE0004220620A494E42204A0A49424220720A70
:101CF0004F4443200E0A49444320060A53444320DC
:101D00001C0A434443202C0A4F5043203C0A5342B0
:101D10004320520A43424320620A494E43204A0A62
:101D200049424320720A4F4444200E0A4944442049
:101D3000060A534444201C0A434444202C0A4F50B2
:101D400044203C0A53424420520A43424420620A3F
:101D5000494E44204A0A49424420720A4F444520D1
:101D60000E0A49444520060A534445201C0A4344B0
:101D700045202C0A4F5045203C0A53424520520A28
:101D800043424520620A494E45204A0A49424520BD
:101D9000720A4F4446200E0A49444620060A53441C
:101DA00046201C0A434446202C0A4F5046203C0A39
:101DB00053424620520A43424620620A494E462078
:101DC0004A0A49424620720A44554D503F0545444F
:101DD000554D8F055644554DD40544535245B70BC8
:101DE0004453434FAE0B44534445A50B494347204E
:101DF000C60A49434520E50A49435020FC0A50578A
:101E00004D38980A50574520AC0A50574F20C20A07
:101E1000444453200F0C424C44526A0D4144432029
:101E2000B40941445220EC0953504D203709535016
:101E30004F204F09535043206509535057208109C3
:101E4000535052208F09535053209B095457492017
:101E5000280854575320E708545750200309545773
:101E600041204B08545757207F0854575220AF0841
:101E700054574220190900000000F93C3DFAF8418E
:101E800074746F424153494320666F722041546D10
:101E900065676133325534FAF85665723A20322E4E
:101EA0003131204275696C6420636F64653A203279
:101EB000303132303330382E30333133FAF93C2D73
:101EC0000000F84F726967696E616C20636F64652A
:101ED00020284329323030322062792052696368E9
:101EE0006172642043617070656C73FAF868747491
:101EF000703A2F2F70726F6A656374732E6361700E
:101F000070656C732E6F7267202070726F6A6563E4
:101F100074734063617070656C732E6F726720FA22
:101F2000F93C2DFAF854686520666F6C6C6F776920
:101F30006E672061726520656E68616E63656D65B0
:101F40006E74732062792053636F747420566974C1
:101F5000616C65FAF86B73765F70726A40676D78D2
:101F60002E636F6D20FAF84D65676138382F313672
:101F7000382F3332382F3332553420706F7274203B
:101F8000284329323031312C3230313220FAF854A2
:101F900057492F5350492F444453202620496E70EF
:101FA000757420436170747572652028432932303E
:101FB000313120FAF84D656761333255342055537D
:101FC0004220262044465520426F6F746C6F616436
:101FD000657220737570706F7274202843293230D7
:101FE000313220FAF93C2DFAF855534220536572EC
:101FF00069616C20492F4F20284329323030382C1A
:102000003230313020504A52432E434F4D2C204C19
:102010004C4320FAF8687474703A2F2F7777772E34
:10202000706A72632E636F6D2F7465656E73792F9E
:1020300020FAF93C2DFAF8416C6C207269676874DB
:102040007320616E642072656D65646965732065D7
:102050007870726573736C792072657365727665DA
:1020600064FAF84E6F7420666F7220636F6D6D6551
:10207000726369616C20757365FAF93C3DFA000082
:10208000F9352DFA00005661726961626C65732042
:10209000696E2052414D3AFA000045455020436F89
:1020A0006E74656E74733AFA000050524F47524195
:1020B0004D204D656D6F727920436F6E74656E743F
:1020C000733AFA0000004E65787420617661696C9D
:1020D00061626C65206C6F636174696F6E3A200099
:1020E0000000FB3A2050726F6772616D20746F6F51
:1020F000206C6172676520666F722045455021FA39
:102100000000536176696E6720746F204545502E3C
:10211000FA000000FB45455020657261736564213B
:10212000FA0000004C6F6164696E672066726F6D23
:1021300020454550FA000000427265616BFA0000CC
:10214000467265653A2070616765733A00002063E6
:10215000686172733A000000FA496E766F6B696EBF
:102160006720626F6F746C6F6164657220617420A8
:10217000307800004572726F72200000FB303A2008
:10218000556E6B6E6F776E20636F6D6D616E642040
:102190006F72206F70657261746F722E0000FB3178
:1021A0003A20456E636F756E7465726564206120B8
:1021B00076616C75652074686174206973206E6F38
:1021C00074206265747765656E203020616E6420CE
:1021D0003235352E0000FB323A2050726F67726143
:1021E0006D206D656D6F72792069732066756C6CFA
:1021F0002E000000FB333A20456E636F756E7465E8
:102200007265642061206368617261637465722025
:1022100074686174206973206E6F74206120726528
:10222000636F676E697A656420747970652E00004B
:10223000FB343A696E7465726E616C206572726F00
:1022400072202D20627566666572206C696D6974F6
:10225000206578636565646564000000FB353A209D
:10226000496E617070726F70726961746520766119
:10227000726961626C65206E616D6520656E636F69
:10228000756E74657265642E0000FB363A204461F9
:10229000746120737461636B20707573682065725C
:1022A000726F72202D20746F6F206D616E792061C6
:1022B0007267756D656E7473206F6E206F6E65202A
:1022C0006C696E652E000000FB373A204461746132
:1022D00020737461636B20706F70206572726F720F
:1022E0002EFAF9092046756E6374696F6E20747258
:1022F00069656420746F2075736520612076616C58
:102300007565207468617420776173206E6F742026
:10231000617661696C61626C652E0000FB383A2061
:102320004D616368696E6520737461636B206572CB
:10233000726F72FAF9092046756E6374696F6E7375
:1023400020616E642F6F722063616C6C73206E6508
:102350007374656420746F6F20646565706C792098
:102360006F7220746F6F20636F6D706C6578000002
:10237000FB393A20474F544F206F7220474F535537
:10238000422064657374696E6174696F6E206C6954
:102390006E6520776173206E6F7420666F756E6452
:1023A0002E000000FB413A20537065636966696541
:1023B000642062697420706F736974696F6E207233
:1023C000616E6765206F6620303A372065786365F7
:1023D000656465640000FB423A204C696E65206EBE
:1023E000756D62657220686173206D6F726520740F
:1023F00068616E207468726565206E756D657261C6
:102400006C730000FB433A2053706563696669652D
:10241000642062697420706F736974696F6E2072D2
:10242000616E6765206F6620303A3120657863659C
:10243000656465640000FB443A2053706563696617
:102440006965642062697420706F736974696F6E66
:102450002072616E6765206F6620303A33206578A0
:102460006365656465640000FB453A20496E7075DC
:102470007420436170747572652072656769737446
:102480006572206F766572666C6F77000000FB46A0
:102490003A2041726974686D65746963206F76656E
:1024A00072666C6F77000000FB31303A2041726930
:1024B00074686D6574696320756E646572666C6FAF
:1024C00077000000FB31313A204469766964652069
:1024D0006279207A65726F000000FB31323A205435
:1024E000574920627573206572726F72206F636343
:1024F000757265640000FB31333A205457492069F6
:102500006E74657266616365206E6F7420656E61BE
:10251000626C65640000FB31343A20545749205303
:102520006C617665207265706C696564207769748A
:1025300068204E414B000000FB31353A204E6F20A1
:10254000426F6F742D6C6F6164657220666F756E7B
:102550006400000000000000000000000000000017
:10256000000000000000000000000000000000006B
:10257000000000000000000000000000000000005B
:10258000000000000000000000000000000000004B
:10259000000000000000000000000000000000003B
:1025A000000000000000000000000000000000002B
:1025B000000000000000000000000000000000001B
:1025C000000000000000000000000000000000000B
:1025D00000000000FFFFFFFFFFFFFFFFFFFFFFFF07
:1025E000FFFFFFFFFFFFFFFFFFFFFFFFFFFFFFFFFB
:1025F000FFFFFFFFFFFFFFFFFFFFFFFFFFFFFFFFEB
:10260000FFFFFFFFFFFFFFFFFFFFFFFFFFFFFFFFDA
:10261000FFFFFFFFFFFFFFFFFFFFFFFFFFFFFFFFCA
:10262000FFFFFFFFFFFFFFFFFFFFFFFFFFFFFFFFBA
:10263000FFFFFFFFFFFFFFFFFFFFFFFFFFFFFFFFAA
:10264000FFFFFFFFFFFFFFFFFFFFFFFFFFFFFFFF9A
:04265000FFFFFFFF8A
:1068000080E090E00895112481E08093D70080EA31
:106810008093D80082E189BD09B400FEFDCF80E9F4
:106820008093D8001092E0001092880A1092890A92
:106830008CE08093E2007894089511241092E20095
:1068400081E08093E0001092D80019BC1092880A71
:1068500080938C0A08958091880A08952FB7F89440
:106860008091880A882369F083E08093E9009BE6A1
:106870008091E80085FD09C082FF03C09093E80085
:10688000F7CF2FBF2FEF3FEF0CC09091F100809119
:10689000E80085FD03C08BE68093E8002FBF292F19
:1068A00030E0C90108952FB7F8948091880A8823B1
:1068B00011F490E010C083E08093E9009091F20021
:1068C000992349F48091E80082FF05C085FD03C04B
:1068D0008BE68093E8002FBF892F08958091880A66
:1068E000882371F09FB7F89483E08093E9002BE64A
:1068F00002C02093E8008091E80085FDFACF9FBF99
:106900000895482F11248091880A8823D9F12FB740
:10691000F89484E08093E90080918B0A882341F009
:106920008091E80085FD02C02FBF12C010928B0A33
:106930009091E400975E34E08091E80085FD13C0FB
:106940002FBF8091E400891729F481E080938B0A9E
:106950008FEF08958091880A8823A1F02FB7F894CB
:106960003093E900E9CF4093F1008091E80085FD84
:1069700003C08AE38093E80085E080938A0A2FBFF2
:1069800080E008958FEF0895282F11248091880AC0
:10699000882351F09FB7F89484E08093E9008091B8
:1069A000E80085FD03C09FBF8FEF08952093F1009D
:1069B0008091E80085FD03C08AE38093E80085E0CC
:1069C00080938A0A9FBF80E0089511249FB7F894AE
:1069D00080918A0A882341F084E08093E9008AE369
:1069E0008093E80010928A0A9FBF08951F920F9229
:1069F0000FB60F9211248F939F938091E100109214
:106A0000E100982F83FF11C01092E90081E080938C
:106A1000EB001092EC0082E18093ED0088E080931F
:106A2000F0001092880A1092890A92FF13C0809198
:106A3000880A882379F080918A0A882359F0815046
:106A400080938A0A882331F484E08093E9008AE302
:106A50008093E8009F918F910F900FBE0F901F9031
:106A600018951F920F920FB60F9211240F931F9338
:106A70002F933F934F935F936F937F938F939F9346
:106A8000AF93BF93EF93FF931092E9008091E800DA
:106A900083FF3CC14091F1003091F1008091F10001
:106AA000682F70E02091F100922F80E0682B792B05
:106AB0008091F100A82FB0E02091F100922F80E0AA
:106AC000A82BB92B1091F1000091F10082EF809377
:106AD000E800363009F05AC02AEA3EE6A9014550DE
:106AE0005040F9013797859194918617970701F5E2
:106AF000FA01859194918A179B07D1F49A012E5F30
:106B00003F4FF901659174912E5F3F4FF901449118
:106B1000212F30E0902F80E0282B392B2F3F31059B
:106B200019F010F02FEF30E0241758F4422F09C06D
:106B3000295F3F4F495F5F4FFEE6243D3F0789F6DF
:106B4000E5C05EEF8091E800282F30E0C901857034
:106B50009070892BB9F322FDDCC0342F413108F04D
:106B600030E1232FCB0106C0FC010196E491E093B4
:106B7000F10021502223C1F7630F711D431B509375
:106B8000E8004423F9F63031E9F2C3C0353061F44E
:106B90008EEF8093E8008091E80080FFFCCF862F85
:106BA00080688093E300B5C0393051F5442309F083
:106BB000ADC06093880A1092890A10928A0A8EEFFB
:106BC0008093E8008DEC9EE621E02093E900FC0133
:106BD0000196E491E093EB00EE2369F0AC014F5F86
:106BE0005F4FFC0184918093EC00CA010196FA0189
:106BF00034913093ED002F5F253039F78EE181C05D
:106C0000383061F4403809F081C08091E80080FF9D
:106C1000FCCF8091880A8093F10050C0313289F412
:106C2000413A09F073C08091E80080FFFCCFE0E8B2
:106C3000FAE081918093F1008AE0E738F807C9F71C
:106C40003DC03032A1F4413209F060C08091E800CB
:106C500082FFFCCFE0E8FAE08091F10081938AE0C6
:106C6000E738F807C9F78BEF8093E80027C0323286
:106C700051F4413209F04AC06093890A8091E800DA
:106C800080FFFCCF1BC03323E9F48091E80080FF34
:106C9000FCCF423811F080E00DC0A093E900809154
:106CA000EB0090E025E0969587952A95E1F78170B5
:106CB0001092E9008093F1001092F1008EEF809322
:106CC000E80027C0313011F0333001F54230F1F4E3
:106CD000672BE1F42A2F2F77822F81508430B0F474
:106CE0008EEF8093E8002093E900333079F089E15A
:106CF0008093EB0081E090E002C0880F991F2A95F5
:106D0000E2F78093EA001092EA0003C081E28093E8
:106D1000EB00FF91EF91BF91AF919F918F917F9188
:106D20006F915F914F913F912F911F910F910F9014
:106D30000FBE0F901F90189500E1000000000800A2
:106D4000FFFFFFFFFFFFFFFFFFFFFFFFFFFFFFFF53
:106D5000FFFFFFFFFFFFFFFFFFFFFFFFFFFFFFFF43
:106D6000FFFFFFFFFFFFFFFFFFFFFFFFFFFFFFFF33
:106D7000FFFFFFFFFFFFFFFFFFFFFFFFFFFFFFFF23
:106D8000FFFFFFFFFFFFFFFFFFFFFFFFFFFFFFFF13
:106D9000FFFFFFFFFFFFFFFFFFFFFFFFFFFFFFFF03
:106DA000FFFFFFFFFFFFFFFFFFFFFFFFFFFFFFFFF3
:106DB000FFFFFFFFFFFFFFFFFFFFFFFFFFFFFFFFE3
:106DC000FFFFFFFFFFFFFFFFFFFFFFFFFFFFFFFFD3
:106DD000FFFFFFFFFFFFFFFFFFFFFFFFFFFFFFFFC3
:106DE000FFFFFFFFFFFFFFFFFFFFFFFFFFFFFFFFB3
:106DF000FFFFFFFFFFFFFFFFFFFFFFFFFFFFFFFFA3
:106E00001201000202000010C0167A040001010203
:106E1000030109024300020100C03209040000011D
:106E200002020100052400100105240101010424CF
:106E3000020605240600010705820310004009042C
:106E40000100020A000000070503024000000705D8
:106E500084024000000403090408034B0053005659
:106E60000000001E034100740074006F00420041E6
:106E7000005300490043002000560033002E0078E4
:106E80000000001E034100740074006F00420041C6
:106E9000005300490043002000560033002E0078C4
:106EA00000000000010000006E1200020000126EDF
:106EB0004300030000556E0401030904596E0802E3
:106EC000030904636E1E03030904836E1E0001C1DF
:086ED00012018036018136FF3A
:00000001FF
